:020000040800F2
:10000000700D002065010008BF110008AD0C00084C
:1000100000000000000000000000000000000000E0
:10002000000000000000000000000000F1170008C0
:100030000000000000000000C5130008351A000889
:1000400077010008770100087701000877010008B0
:10005000770100087107000877010008950700087C
:10006000770100087701000877010008ED05000816
:100070007701000877010008770100087701000880
:1000800077010008770100080000000077010008F0
:100090007701000877010008770100087701000860
:1000A000770100087701000877010008D91A0008D5
:1000B0007701000800000000770100080000000040
:1000C00000F002F800F03EF80CA030C80838241800
:1000D0002D18A246671EAB4654465D46AC4201D180
:1000E00000F030F87E460F3E0FCCB6460126334274
:1000F00000D0FB1AA246AB46334318471C28000029
:100100003C280000103A02D378C878C1FAD85207C8
:1001100001D330C830C101D504680C6070470000BD
:100120000023002400250026103A01D378C1FBD813
:10013000520700D330C100D50B6070471FB51FBDFB
:1001400010B510BD00F01CF91146FFF7F7FF01F0E4
:100150009DFF00F034F903B4FFF7F2FF03BC00F099
:100160003BF900000748804707480047FEE7FEE7E5
:10017000FEE7FEE7FEE7FEE704480549054A064BB1
:10018000704700005D1A0008C100000870070020D9
:10019000700D0020700900207009002030B5441C4B
:1001A00003E00178401C00290DD08107F9D10B4BE9
:1001B000DD0104C8D11A91432940FAD0001B0A0678
:1001C00003D0C01E30BD001B30BD0A0401D0801E0C
:1001D00030BD0902FCD0401E30BD0000010101010C
:1001E00001E004C0091F0429FBD28B0701D502805E
:1001F000801CC90700D00270704700290BD0C307CC
:1002000002D00270401C491E022904D3830702D584
:100210000280801C891EE3E70022EEE70022DFE770
:10022000002203098B422CD3030A8B4211D30023F3
:100230009C464EE003460B433CD4002243088B42CD
:1002400031D303098B421CD3030A8B4201D394465A
:100250003FE0C3098B4201D3CB01C01A524183094D
:100260008B4201D38B01C01A524143098B4201D307
:100270004B01C01A524103098B4201D30B01C01A32
:100280005241C3088B4201D3CB00C01A52418308AC
:100290008B4201D38B00C01A524143088B4201D3D9
:1002A0004B00C01A5241411A00D201465241104639
:1002B00070475DE0CA0F00D04942031000D34042AE
:1002C000534000229C4603098B422DD3030A8B42E4
:1002D00012D3FC22890112BA030A8B420CD3890182
:1002E00092118B4208D3890192118B4204D3890168
:1002F0003AD0921100E08909C3098B4201D3CB01A6
:10030000C01A524183098B4201D38B01C01A52415A
:1003100043098B4201D34B01C01A524103098B425E
:1003200001D30B01C01A5241C3088B4201D3CB0049
:10033000C01A524183088B4201D38B00C01A52412C
:10034000D9D243088B4201D34B00C01A5241411A03
:1003500000D20146634652415B10104601D3404231
:10036000002B00D54942704763465B1000D34042E2
:1003700001B50020C046C04602BD704770477047B7
:10038000754600F025F8AE46050069465346C0089C
:10039000C000854618B020B5FFF7EEFE60BC002710
:1003A0004908B6460026C0C5C0C5C0C5C0C5C0C541
:1003B000C0C5C0C5C0C5403D49008D46704710B599
:1003C0000446C046C0462046FFF7C5FE10BD0000EB
:1003D000004870470C07002001491820ABBEFEE71B
:1003E000260002007047000038B50021009100246B
:1003F0006A460F4801F088FC68460078002815D14D
:1004000001F090FE002811D000BF0CE0204601F062
:1004100095FE002805D0E100064A89184868804703
:1004200003E0601CC4B20E2CF0DB00BF38BD00003E
:10043000700600202C2800080548008805498842DD
:1004400004D003480088401C014908807047000020
:1004500062000020FFFF000010B5002000F0F6FE53
:1004600004462078042805DA608822789200124B2E
:100470009958884711480078401C10490870084670
:100480000078322802DD642008700BE00B48007809
:100490000A2807DD6420094908700022032110465C
:1004A00000F020FF064800887D210901884202DB18
:1004B00000200349088010BD9C2800087800002017
:1004C0006200002010B50024542200210C4800F0E6
:1004D0006BFE0C48007800060A4949780904084375
:1004E00008498978090208430649097908430446FE
:1004F000204600F0DDFB02494031888110BD00003C
:10050000B80600200033000810B53448C07901282F
:1005100022D133480078401C3149087008460078E1
:10052000052804DA10212F4800F056FA21E02C4863
:100530000078092807DB0020294908701021294884
:1005400000F048FA15E026480078052811DD102152
:10055000244800F03FFA0CE02048C079022804D17A
:100560001021204800F038FA03E010211D4800F067
:1005700031FA1A48007A012822D11B480078401C21
:100580001949087008460078052804DA082115483A
:1005900000F022FA21E014480078092807DB002047
:1005A0001149087008210F4800F014FA15E00E48B0
:1005B0000078052811DD08210A4800F00BFA0CE04C
:1005C0000648007A022804D10821064800F004FAFF
:1005D00003E00821034800F0FDF910BDF8060020F3
:1005E0005A000020000400485B00002010B50120E4
:1005F000800300F0D7F8002803D00120800300F02A
:10060000CBF810BD10B55748807D002804D180215B
:10061000554800F0DFF92EE05248807D012804D1D2
:100620008021514800F0D8F925E04E48807D02280D
:1006300021D14E480078401C4C490870084600788B
:10064000052804DA8021484800F0C6F913E047483D
:100650000078092807DB00204449087080214248BF
:1006600000F0B8F907E041480078052803DD802153
:100670003D4800F0AFF93B4816304078002804D1DF
:100680004021394800F0A6F930E03648163040786D
:10069000012804D14021344800F09EF926E0314879
:1006A00016304078022821D130484078401C2F492C
:1006B000487008464078052804DA40212A4800F0AE
:1006C0008BF913E029484078092807DB00202749E7
:1006D00048704021244800F07DF907E02348407825
:1006E000052803DD4021204800F074F91D4816302C
:1006F0008078002804D120211B4800F06BF930E0FD
:10070000184816308078012804D12021164800F0BE
:1007100063F926E0134816308078022821D1134867
:100720008078401C1149887008468078052804DAD2
:1007300020210D4800F050F913E00C48807809287A
:1007400007DB0020094988702021074800F042F9A2
:1007500007E006488078052803DD2021024800F0E4
:1007600039F910BDD80600200004004856000020CA
:1007700010B5012000F016F8002802D0012000F08A
:100780000BF8022000F00EF8002802D0022000F042
:1007900003F810BD70470000014948617047000030
:1007A0000004014001460020044A52690A40002A20
:1007B00001D0012000E0002070470000000401404B
:1007C000002120498279002A35D00A461268036840
:1007D0009A430B461A600A46526803689A430B46CE
:1007E0005A60027951180A6803681A430A60154A68
:1007F000926803689A43134B9A601A46D26803685A
:100800009A43104BDA604279102A0CD11A4692684A
:1008100003681A430B4B9A601A46D26803681A435E
:10082000084BDA600DE00749427951180A680368FD
:100830001A430A6005E0027951180A6803689A436E
:100840000A6070470004014000B585B001214804EA
:1008500000F07AFE0121880500F076FE01210846AD
:1008600000F092FE01208002009001216846017193
:10087000002181710121C17169460920C00600F083
:1008800035F8012189020920C00600F0A5F80120F1
:10089000009000216846017101218171032141719D
:1008A0000121C17169460F4800F020F800210520A0
:1008B00000F0A0FF012003900021684601740C2184
:1008C00041740121817403A8FFF77AFF052168466E
:1008D0000172002141720121817202A800F070FCB6
:1008E00005B000BD0014004870477047F0B50A46D7
:1008F00000210023002400BF3DE001258D402B4650
:1009000015681D402C469C4234D11579012D02D02A
:100910001579022D16D185684F000326BE40B543D8
:10092000856055794E00B540866835438560858879
:1009300001268E40B5438580858896798E40B6B273
:100940003543858005684F000326BE40B5430560EA
:1009500015794E00B540066835430560C5684F00FF
:100960000326BE40B543C560D5794E00B540C66884
:100970003543C560491C1029BFD3F0BDF0B5002335
:1009800000244D07EE0E1546B5402B46CD10AE00A7
:1009900005462035AD594E07F70E0F26BE40B5432C
:1009A000CE10B60007462037BD51CD10AE003D46F3
:1009B000AD591D432C46CD10AD003E467451F0BDDF
:1009C00002460020138A0B40002B01D0012000E0DA
:1009D0000020704701857047816170471CB5012177
:1009E0000720400400F0B0FD0121880500F0ACFDB7
:1009F0000121084600F0C8FD012000900121684651
:100A0000017103214171002181710121C171694688
:100A10000920C006FFF76AFF1020009001216846F8
:100A2000017103214171002181710121C171694668
:100A30000920C006FFF75AFF10210920C006FFF762
:100A4000C9FF2020009000216846017101218171B9
:100A5000032141710121C17169460920C006FFF7D8
:100A600045FF002206210920C006FFF787FF40202E
:100A700000900221684601710321417100218171BA
:100A800069460920C006FFF731FF40200090012190
:100A90006846017103214171002181710121C171F9
:100AA00069460920C006FFF721FF40210920C00642
:100AB000FFF792FF8020009000216846017101211C
:100AC0008171032141710121C17169460920C0066C
:100AD000FFF70CFFFF2001300090002168460171F4
:100AE00001218171032141710121C17169460920F0
:100AF000C006FFF7FBFE012000900021684601714F
:100B000001218171032141710121C171694666484A
:100B1000FFF7ECFE022000900021684601710121E0
:100B20008171032141710121C17169465E48FFF75E
:100B3000DDFE012040020090002168460171012184
:100B40008171032141710121C17169460920C006EB
:100B5000FFF7CCFE01208002009000216846017161
:100B600001218171032141710121C171694609206F
:100B7000C006FFF7BBFE0120C002009000216846BE
:100B8000017101218171032141710121C171694606
:100B90000920C006FFF7AAFE0120000300900021F3
:100BA0006846017101218171032141710121C171E7
:100BB00069460920C006FFF799FE0120C003009096
:100BC00001216846017103214171002181710121D8
:100BD000C17169460920C006FFF788FE0121C903DB
:100BE0000920C006FFF7F6FE0820009001216846A4
:100BF000017103214171002181710121C171694697
:100C00002948FFF773FE08212748FFF7E3FE10206D
:100C10000090012168460171032141710021817119
:100C20000121C17169462048FFF760FE10211E486E
:100C3000FFF7D0FE202000900121684601710321BA
:100C40004171002181710121C17169461648FFF788
:100C50004DFE20211448FFF7BDFE402000900121E9
:100C60006846017103214171002181710121C17127
:100C700069460D48FFF73AFE40210B48FFF7AAFEF0
:100C800080200090012168460171032141710021FB
:100C900081710121C17169460348FFF727FE802158
:100CA0000148FFF797FE1CBD0004004800BFFEE7A7
:100CB0000246002100202A4B1B78302B08DB284BF2
:100CC0001B78392B04DC264B1B78303B99B203E0B0
:100CD000234B1B78373B99B20B07180C204B5B78E2
:100CE000302B08DB1E4B5B78392B04DC1C4B5B780C
:100CF000303B99B203E01A4B5B78373B99B20B0655
:100D0000190C03460B431846154B9B78302B08DB18
:100D1000134B9B78392B04DC114B9B78303B99B2F9
:100D200003E00F4B9B78373B99B20B05190C034638
:100D30000B4318460A4BDB78302B08DB084BDB787B
:100D4000392B04DC064BDB78303B99B203E0044BD3
:100D5000DB78373B99B203460B43184670470000D7
:100D6000003300080148024908607047CCCC0000FD
:100D7000003000400148024908607047AAAA0000FC
:100D800000300040014948607047000000300040DA
:100D90000149886070470000003000400149086048
:100DA000704700000030004010B524480078401C17
:100DB0002249087022480078401C214908702148C7
:100DC0000088401C1F4908801F480088401C1E499D
:100DD0000880FF2101310920C006FFF7F1FD00283E
:100DE00007D1174800780F280DDB00201449087040
:100DF00009E0002013490880114908701348008851
:100E0000401C124908800F4800887D210901884252
:100E100006DD00200B4908800D4A012100F062FA2E
:100E20000A4800880B49884207D1002007490880FA
:100E3000074A521E012100F055FA10BD1C00002087
:100E40001D000020200000201E00002022000020A5
:100E5000040700003075000010B526480078401CDB
:100E60002449087024480078401C2349087023480E
:100E70000088401C2149088021480088401C2049E6
:100E8000088001211F48FFF79BFD002812D11A4856
:100E900000780A2805DB00201749087001211A484C
:100EA000C17300201549088018480088401C174964
:100EB000088005E000201049087000211248C17325
:100EC0000E4800881249884206DD00200B49088040
:100ED000104A012100F006FA0C4800880E498842A9
:100EE00007D10020094908800A4A521E012100F05A
:100EF000F9F910BD14000020150000201800002092
:100F00001600002000040048F80600201A00002007
:100F1000E02E000004060000307500001CB500241F
:100F2000002000900190012189020920C006FFF7EE
:100F300047FD002801D1012100E000216846017031
:100F40008848C17B6846417080210920C006FFF7B0
:100F500037FD002801D1012000E00020694688709B
:100F6000012109030920C006FFF72AFD002801D14D
:100F7000012000E000206946C8700121C902092053
:100F8000C006FFF71DFD002801D1012000E0002070
:100F90006946087102217448FFF712FD002801D14B
:100FA000012000E000206946487101214902092022
:100FB000C006FFF705FD002801D1012100E0002156
:100FC0006846817120210920C006FFF7F9FC01461F
:100FD0006846C1714079002824D0684640780028CE
:100FE00020D062480078401C6049087008460078AC
:100FF000032809DD5E480078002805D101205C49FE
:10100000087000205949087059480078012808D113
:101010000220574908700D2212020121002000F021
:1010200061F91CBD00205149087051480078022820
:1010300008D1504A0121002000F054F900204C4909
:101040000870EEE700204A490870002484E06846F2
:10105000005D002831D143482038C07F0121A140E4
:10106000884340492039C877002043490855434800
:10107000005D401C4149085501204149087000208D
:101080006100404A50523D48005D032862DD002067
:101090003A4908553C48005D6946095D884259D087
:1010A000601D0002401C82B20121002000F01AF9EC
:1010B0006846005D344908554CE02A482038C07F16
:1010C0000121A1400843C1B226482038C1772A48EF
:1010D000005D401C2849085500202849085560003B
:1010E0002849085A401C6100264A50522248005D97
:1010F00003282FDD00202049085560001146085ABA
:10110000322816DD0020610050521D480078022868
:1011100020D002201A490870012C1BD0022C19D0B3
:10112000601D0002801C82B20121002000F0DAF86C
:1011300010E01548005D6946095D88420AD0601DCF
:101140000006020C0121002000F0CCF86846005D8A
:101150000D490855601CC4B2082C00DA77E700BFBF
:101160005FE70000F806002000040048440000206B
:1011700045000020010D0000340000203C0000204C
:10118000460000208C000020240000207047000052
:1011900010B50449887C00F0B9FBFFF733FAFFF77C
:1011A000B3F910BDD806002030B50446002303E093
:1011B0002170641C5D1CABB29342F9DB30BD7047FB
:1011C00000218278002A27D0184A03231B02D21854
:1011D00003789B109B00D15802789207D30EFF2210
:1011E0009A400B469343194642789207120E0378B1
:1011F0009B07DB0E9A4011430C4A03231B02D218B3
:1012000003789B109B00D1500278D306DB0E01229D
:101210009A40064B1A6007E00278D306DB0E0122E3
:101220009A40024B80331A607047000000E100E0F2
:10123000002252214143044B5A54802252214143FF
:10124000C9184A70704700009C00002070B5014624
:1012500000201C4D2870522048431B4D285C43063B
:101260005B0E52204843401940784206520E5220ED
:10127000484340194078802528400446002C13D16B
:1012800052204843104D4019801C950040190D4DC7
:1012900006882E8040886880501CC2B2142A00DB69
:1012A0000022934200D10124002C01D0802002436F
:1012B00052204843044D2B54522048434019427059
:1012C000004870BD480000209C00002010B500249C
:1012D00004E02046FFF7ACFF601CC4B2072CF8DB2B
:1012E00010BD0000F8B50B466E4633707280522672
:1012F00046431A4FBE5D7106490E52264643BE5DF7
:1013000080273E40354652264643144FF6197678DC
:101310007406640E002D13D152264643F619B61CEE
:101320008F00F7196E4636883E806E4676887E803E
:101330004E1CF1B2142900DB0021A14200D101258D
:10134000002D01D08026314352264643034FB95524
:1013500052264643F6197470F8BD00009C00002028
:1013600010B502460020154B18688008800003461F
:1013700013431846114B1860114B1B690424234377
:101380000F4C2361012907D130BF23461B69042478
:10139000A3430B4C23610FE0022907D120BF084B68
:1013A0001B690424A343064C236105E0044B1B691D
:1013B00002242343024C236110BD00000070004052
:1013C00000ED00E07047000010B5474800780300CA
:1013D00000F0D6FD09060E1D2A323B47485587000E
:1013E00041480078401C404908700020488079E05E
:1013F0003D4840887D21C900884200DC72E0002021
:101400003949488008460078401C08706AE0364830
:1014100040887D210901884200DC63E03248007881
:10142000401C314908705DE000202F494880084683
:101430000078401C087055E000202B49C880488087
:1014400008460078401C08704CE02748408827492F
:10145000884200DC46E024480078401C224908709D
:1014600040E03FE0204840887D21C900884200DC00
:1014700038E000201C4948800820087032E01A48F3
:101480004088642800DA2DE0FFF7DEF900F0D6FA94
:1014900000F0E4FA0120164948707D21C900154882
:1014A0000068FEF7BDFE0446601E1349884201D95C
:1014B00001200CE0601E114948610321081F00F063
:1014C0006DFD00200D49886107200861002000287B
:1014D00001D000BFFEE705200349087000204880C6
:1014E00000E000BF00BF10BDDC0200208813000038
:1014F000B806002000000020FFFFFF0000E000E031
:101500000A4840880A49884204D008484088401C5C
:10151000064948800548C0880549884204D00348E8
:10152000C088401C0149C88070470000DC020020D0
:10153000FFFF0000002003490870488008718860A0
:10154000C8807047DC020020002905D0054A526996
:101550000243044B5A6104E0024A52698243014B40
:101560005A61704700100240002905D0054AD2692F
:101570000243044BDA6104E0024AD2698243014B20
:10158000DA61704700100240002905D0054A9269CF
:101590000243044B9A6104E0024A92698243014B80
:1015A0009A61704700100240FEB5044600250026EF
:1015B00000200290019000900027864840680C218E
:1015C00008400546002D06D0042D07D0082D08D070
:1015D0000C2D2CD128E0804820602BE07E48206034
:1015E00028E07C4840680F21890408400646794875
:1015F00040680321C90308400290B00C861C029881
:10160000002803D17548374647430BE07148C06A4C
:101610000007000F401C01906F480199FEF700FE83
:1016200070430746276005E06D48206002E06A4885
:10163000206000BF00BF67484068F02108400546B1
:101640002D096848405D009020680099C84060609E
:101650006048406807210902084005462D0A614894
:10166000405D009061680098C140A1605948006BDE
:10167000FF2101310840884202D05B48E0600DE064
:1016800054484068012189030840884203D0A0687B
:101690004008E06002E0A0688008E0604D48006B10
:1016A00040210840402802D05048206102E001203B
:1016B000C00320614748006B10210840102802D069
:1016C0004548606101E0206860614248006B800726
:1016D000800F002802D1A068A06119E03D48006B8E
:1016E0008007800F012802D12068A06110E03948EE
:1016F000006B8007800F022802D18003A06107E001
:101700003448006B8007800F032801D13248A06164
:101710003048006B032109040840002802D1A0686A
:10172000E06120E02B48006B0321090408400121FF
:101730000904884202D12068E06114E02548006B6A
:1017400003210904084001214904884202D1801084
:10175000E06108E01F48006B03210904084088424B
:1017600001D11D48E0611B48006B0321890408403A
:10177000002802D1A068206220E01648006B0321F7
:101780008904084001218904884202D1206820622E
:1017900014E01048006B0321890408400121C904AA
:1017A000884202D10011206208E00A48006B032140
:1017B00089040840884201D1074820620548006B2F
:1017C00080210840802802D00548606200E06762FE
:1017D000FEBD00000010024000127A0000093D002A
:1017E000006CDC0279000020809FD5001280000090
:1017F0007047000030B500228B071C0F0F23A34059
:101800001A460B4B8C10A4001B599343084C8D10A7
:10181000AD00635123468C10A4001B598C07250F83
:101820000446AC402343024C8D10AD00635130BDE3
:10183000080001400CB5002001900090304800687D
:101840000121090408432E49086000BF2C480068A4
:1018500001214904084000900198401C0190009823
:10186000002803D1274901988842EFD12448006815
:10187000012149040840002802D00120009001E025
:10188000002000900098012839D111201E490860DD
:101890001B4840681A494860084640684860084646
:1018A00040687F21C903884315494860084640685D
:1018B00011210904084312494860084600680121C3
:1018C000090608430E49086000BF0D480068012161
:1018D000490608400028F8D0094840688008800080
:1018E00007494860084640680221084304494860A7
:1018F00000BF034840680C2108400828F9D10CBDFE
:1019000000100240FFFF00000020024010B5044616
:10191000002C05D140210920C006FFF75BF82EE01E
:10192000012C05D140210920C006FFF755F826E01B
:10193000022C24D112480078401C11490870084636
:101940000078052805DA40210920C006FFF744F891
:1019500015E00B480078092808DB40210920C00663
:10196000FFF738F800200649087008E004480078BE
:10197000052804DD40210920C006FFF72BF810BD23
:1019800055000020002106E0064900BF0A464B1E14
:1019900099B2002AFAD10246431E98B2002AF3D126
:1019A000704700003818000010B51C480078FF2868
:1019B00004D01A480078401C18490870184800786C
:1019C000FF2804D016480078401C154908701548B7
:1019D0000078FF2804D013480078401C1149087093
:1019E00011480078FF2804D00F480078401C0E49A9
:1019F00008700E48807BFF2805D00C48807B401C77
:101A0000C1B20A488173FFF77BFDFEF715FD084858
:101A10000078401C0649087010BD000050000020EE
:101A2000510000205200002053000020F806002042
:101A30005400002010B5FFF7B7FF10BD10B500200F
:101A400005490861886101210807FFF78DFD012123
:101A50000846FFF785FC10BD00E000E010B51B480C
:101A60000068012108431949086008464068184980
:101A7000084016494860084600681649084013495E
:101A80000860084600680121890488430F490860FE
:101A9000084640683F21090488430C4948600846CD
:101AA000C06A00090001C8620846006BFF2154317A
:101AB0008843064908630846406B40084000486375
:101AC00000208860FFF7B6FE10BD00000010024045
:101AD0000CB8FFF8FFFFF6FE10B500F047F910BD97
:101AE00001627047002904D0026801231A43026092
:101AF00003E002685208520002607047024600206C
:101B0000D3690B40002B01D0012000E0002070477A
:101B1000F8B503460024002600960025002018464C
:101B20000E04340ECEB200960127009EB7403D460B
:101B3000022C01D1001D02E0032C00D10830002A44
:101B400003D006682E43066002E00668AE430660D6
:101B5000F8BD0000F0B58BB004460D46002700200C
:101B60000A90002620684008400020606668032133
:101B70000903304688430646A8680643666026681F
:101B80002D480640E9686868084329690843064308
:101B90002660A66803210902304688430646686924
:101BA0000643A6606846FFF7FFFC2448844202D142
:101BB00006980A900DE02248844202D107980A90C4
:101BC00007E02048844202D108980A9001E0029878
:101BD0000A9020680121C903084000280CD0296818
:101BE0000A9A5000FEF71CFB074629680A9A500023
:101BF000FEF716FB0E4609E029680A98FEF710FB6F
:101C0000074629680A98FEF70BFB0E46286840082D
:101C1000B04200D87F1C20680121C9030840002879
:101C200006D03807460F3846074908403043074674
:101C3000A7810BB0F0BD0000F3E9FFFF00380140C1
:101C40000044004000480040F0FF00000146888C3E
:101C5000C005C00D7047CA05D20D0285704700004F
:101C600000B589B0182101A8FEF7D8FA00F014FBDE
:101C700001214804FFF768FC01218803FFF784FC79
:101C8000012202210920C006FEF778FE012203216D
:101C90000920C006FEF772FE0C200790022108A85A
:101CA00001700321417001218170C17007A90920D1
:101CB000C006FEF71BFEE1204002019000200290CA
:101CC0000390049006900C20059001A90B48FFF7A3
:101CD00041FF01210948FFF705FF01220849074894
:101CE000FFF716FF012207490448FFF711FF4021C3
:101CF0000248FFF7F5FE09B000BD000000380140C2
:101D00000501050006010600F7B50546164C00F072
:101D1000B7FA002824D160784101201D465C1E2EB0
:101D200000DD1E262E706D1C701CC6B2002709E057
:101D300060784101201D0918781C085C28706D1C12
:101D4000781CC7B2B742F3DB6078401C60706078E3
:101D5000142801DB0020607000210298017002E06D
:101D6000022102980170FEBDEC02002070B5002532
:101D7000464C40214648FFF7C1FE002839D00520D7
:101D8000C00120180079002827DD0520C001201897
:101D90000079401E0521C901611808710520C001A4
:101DA00020188079FA2804DB00200521C901611878
:101DB00088710520C001201882790520C0012018F3
:101DC0008079401C0523DB01E31898713148201805
:101DD000815C2F48FFF73FFF07E00520C001201876
:101DE00040790521C9016118887140212848FFF711
:101DF00077FE20212648FFF781FE002844D02448A2
:101E0000FFF724FFC5B224480078002802D001283B
:101E100031D107E0242D02D101201F490870012093
:101E2000E0702CE0232D17D1232120784201201DC2
:101E30001018E2788154E17820784201201D815405
:101E40002078401C20702078142801DB00202070AE
:101E50000020114908700DE0242D02D10120E0700E
:101E600008E020784101201D0818E1784554E07809
:101E7000401CE07003E000200749087000BF00BF6D
:101E800020210348FFF72CFE70BD0000EC0200206B
:101E9000003801408702000060000020F8B50546C8
:101EA0000E46344C002E01D10420F8BD00F0E8F9B4
:101EB000074625E00520C00120180079401C0521B7
:101EC000C901611808710520C00120184079FA285D
:101ED00004DB00200521C90161184871287805211B
:101EE000C901611849790522D201A2185279521C00
:101EF0000523DB01E3185A711F4AA21850546D1CC8
:101F00003046711ECEB20028D4D1002F30D005202B
:101F1000C00120180079002808D00520C001201831
:101F20000079401E0521C901611808710520C00112
:101F300020188079FA2804DB00200521C9016118E6
:101F400088710520C001201880790522D201A218CD
:101F50009279521C0523DB01E3189A71064AA218F4
:101F6000115C0648FFF777FE08210448FFF7B8FD2B
:101F700000209AE7EC0200208702000000380140B0
:101F800030B47446641E2578641CAB4204D3635D90
:101F90005B00E31830BC18471D46F8E710B5002871
:101FA00019DB1A4A03231B02D21883089B00D2585C
:101FB0008307DC0EFF23A3409A438B071B0E840785
:101FC000E40EA3401A43114B032424021B19840876
:101FD000A4001A5118E00E4A03071B0F083B9B0888
:101FE0009B00D2588307DC0EFF23A3409A438B0744
:101FF0001B0E8407E40EA3401A43054B0407240F6D
:10200000083CA408A4001A5110BD000000E100E043
:102010001CED00E010B5002819DB1A4A03231B024F
:10202000D21883089B00D2588307DC0EFF23A340FD
:102030009A438B071B0E8407E40EA3401A43114BEF
:10204000032424021B198408A4001A5118E00E4A24
:1020500003071B0F083B9B089B00D2588307DC0E2D
:10206000FF23A3409A438B071B0E8407E40EA34073
:102070001A43054B0407240F083CA408A4001A5176
:1020800010BD000000E100E01CED00E02048FFF77B
:1020900079FC00F0D7F800F0AFF800F093F800F00A
:1020A00081F800F06DF832E0FEF764FE1948007820
:1020B000052809DB002017490870FEF7CDF9FEF767
:1020C000CBFEFEF771FE22E013480078232807DBE1
:1020D000002011490870FEF787F9FEF71FFF16E090
:1020E0000E480078642809DB00200C490870FFF7CF
:1020F0006BF9FEF7F9FBFFF74BF808E008480078AA
:10210000232803DB00200649087000E000BFCBE76E
:10211000C05D00005000002051000020520000204F
:1021200053000020002104480178405C232801D19D
:10213000012070470020FCE77006002070B50546BE
:1021400000240026E9000C4A5058FEF727F8C6B2D2
:1021500000BF0CE0E80008490858015D601C074A10
:10216000105C814201D0002070BD601CC4B2B4423A
:10217000F0DB0120F8E700002C28000870060020A2
:1021800010B50748FEF70AFE0520FEF7FBFD7D208F
:10219000C000FEF7FDFDFEF7EDFDFEF7E3FD10BD0F
:1021A0005555000000B58BB001A8FFF7FDF90121DE
:1021B000684641701B21017001218170FFF700F812
:1021C0000BB000BD10B50024FEF708FCFFF748FD7A
:1021D00006480468002C07D00548844204D02046F5
:1021E000FEF766FD0349888110BD0000003300083A
:1021F000FFFFFF00F806002010B57D21C9000E4842
:102200000068FEF70DF80446601E0C49884201D9AB
:1022100001200CE0601E0A4948610321081FFFF7F6
:10222000F9FE002006498861072008610020002887
:1022300001D000BFFEE710BD00000020FFFFFF003F
:1022400000E000E010B50020094908700949087055
:102250000949087009490870FFF76CF9FEF796FF05
:10226000FEF730F9FEF741FBFFF730F810BD000034
:102270005000002051000020520000205300002098
:102280000448007803494978884201D10120704709
:102290000020FCE7EC02002003480021017041709F
:1022A0008170C17070470000EC02002010B50A4830
:1022B0004079492805D1002202211046FFF712F883
:1022C00008E005484079562804D100220321104631
:1022D000FFF708F810BD0000700600200648407A9D
:1022E0003038C1B20548C1710348807A3038C1B274
:1022F000024801727047000070060020F8060020B6
:102300000A48407A3038C1B2094881750748807A56
:102310003038C1B20648163041700448C07A3038AF
:10232000C1B203481630817070470000700600206B
:10233000D8060020704710B5002202211046FEF793
:10234000D1FF10BD7047000010B50A48807A3028D0
:1023500005D110210920C006FEF73CFB08E0054826
:10236000807A312804D110210920C006FEF734FB01
:1023700010BD00007006002010B58D48407930383F
:102380000300FFF7FDFD05043A70A6DC390088491B
:10239000C97930390A225143854A127A303A89186C
:1023A00008026421FDF746FFC1B28248C17280492C
:1023B000497A30390A2251437D4A927A303A891853
:1023C00008026421FDF736FFC1B27A4801737849EB
:1023D000C97A30390A225143754A127B303A89183A
:1023E00008026421FDF726FFC1B272488172007CA9
:1023F000012108436F490874D7E06D49C979303924
:102400000A2251436A4A127A303A89180802642132
:10241000FDF710FFC1B2674881736549497A3039C9
:102420000A225143624A927A303A8918080264219A
:10243000FDF700FFC1B25F48C1735D49C97A303909
:102440000A2251435A4A127B303A89180802642101
:10245000FDF7F0FEC1B257484173007C02210843EA
:1024600054490874A1E05249C97930390A225143CC
:102470004F4A127A303A891808026421FDF7DAFED1
:10248000C1B24C4881704A49497A30390A225143D5
:10249000474A927A303A891808026421FDF7CAFE49
:1024A000C1B24448C1704249C97A30390A22514305
:1024B0003F4A127B303A891808026421FDF7BAFEC0
:1024C000C1B23C484170007C04210843394908747A
:1024D0006BE03749C97930390A225143344A127ABC
:1024E000303A891808026421FDF7A4FEC1B23148D0
:1024F00041712F49497A30390A2251432C4A927A44
:10250000303A891808026421FDF794FEC1B22948C7
:1025100081712749C97A30390A225143244A127BF2
:10252000303A891808026421FDF784FEC1B22148BF
:102530000171007C082108431E49087435E01C49DC
:10254000C97930390A225143194A127A303A891826
:1025500008026421FDF76EFEC1B2164801721449EB
:10256000497A30390A225143114A927A303A89180D
:1025700008026421FDF75EFEC1B20E4841720C49AB
:10258000C97A30390A225143094A127B303A8918F4
:1025900008026421FDF74EFEC1B20648C171007CFD
:1025A000102108430349087400BF00BF10BD00009C
:1025B00070060020D806002010B500241648807947
:1025C0003038C4B2002C18D11348017A1348C174B2
:1025D000C07C302806D10121C9030920C006FEF7BE
:1025E000F9F917E00D48C07C312813D10121C90346
:1025F0000920C006FEF7F0F90CE0012C05D10648D1
:10260000017A06481330417004E00348017A034818
:102610001330817010BD000070060020D806002025
:102620000B484079302803D100210A4841740EE05C
:1026300007484079312803D101210648417406E05A
:1026400003484079322802D1022102484174704780
:1026500070060020D80600200020024908700249B8
:1026600048707047DC020020B806002000200249B4
:102670000870024948707047DC020020B80600204C
:102680000020054989793039C8B2022800DD0220CE
:10269000024988747047000070060020D8060020A8
:1026A00070B50646002400250E4C24202070641CC2
:1026B00049202070641C44202070641C2C20207051
:1026C000641C00BF01E0681CC5B20F2DFBDB31208C
:1026D0002070641C23202070641C15210148FFF722
:1026E000DDFB70BD8E06002070B505460024324C1F
:1026F00024202070641C4B202070641C4520207016
:10270000641C59202070641C2812082803D13B2027
:102710002070641C2DE02812092803D13C20207071
:10272000641C26E028120A2803D13D202070641C76
:102730001FE028120B2803D13E202070641C18E0F3
:1027400028120D2803D13F202070641C11E02812AC
:102750000C2803D140202070641C0AE028120E28A7
:1027600003D138202070641C03E028123030207020
:10277000641C2C202070641C012110484172281216
:10278000052807DAE8B2022804D1FF20000205403C
:1027900001200543284630302070641C232020701F
:1027A000641C00202070641C09210348FFF776FB9D
:1027B00000210248817370BD8E060020F8060020BB
:1027C00000BF704770B50646002400250F4C24203A
:1027D0002070641C56202070641C2C202070641C07
:1027E00000BF05E00A48405D2070641C681CC5B24B
:1027F0000F2DF7DB46202070641C23202070641C02
:1028000014210248FFF74AFB70BD00008E0600202D
:1028100014280008535A44313031303132343035C5
:10282000323631002448454152540000082900083E
:1028300035230008F028000859260008D42800088D
:102840006D260008AC28000845230008B8280008B9
:1028500079230008C82800088126000810290008EC
:10286000B9250008EC28000821260008D028000817
:1028700037230008C028000801230008B0280008FA
:10288000DD220008E0280008AD220008FC2800082E
:1028900049230008E428000835230008C127000860
:1028A000E9260008A1260008C52700084D49430075
:1028B00043414C4C4C4544004E4C45440000000004
:1028C000444F4F524C454400554C454400000000D5
:1028D00049440000535953555044415445000000A9
:1028E00041534B0043414C4C000000005349500001
:1028F0005359535245534554000000004E4554521D
:102900004553455400000000484541525400000022
:1029100052454C41590000000833000800000020D7
:102920008C00000004010008943300088C00002093
:10293000E40C00002001000800000000000000007E
:102940000000000000000000000000000000000087
:102950000000000000000000000000000000000077
:102960000000000000000000000000000000000067
:102970000000000000000000000000000000000057
:103300004633303100000000006CDC020000000099
:103310000000000001020304060708090000000085
:10332000000000000000000000000000000000009D
:10333000000000000000000000000000000000008D
:10334000000000000000000000000000000000007D
:10335000000000000000000000000000000000006D
:10336000000000000000000000000000C0A801D321
:10337000C0A801010000C0A801AA000000000000D0
:103380000000000000010203040102030406070814
:043390000900000030
:04000005080000C12E
:00000001FF
